:102227002020202020202020202020200D0A002AE6
:102237004D3A2053656C6674657374206F6B0D0A95
:10224700002A573A2053656C66746573742066617B
:10225700696C65640D0A002A52454144590D0A000C
:1022670000022F002F2A00AB20015E1601D21102B7
:102277005A0C02780B02960A02B60902D70802F92D
:1022870007031C06033F05036404038B0303B20221
:0622970003DA010404005B
:1013EE00906F137401F0906F13E0FD64126024EDA2
:1013FE0075F003A42467F582E43422F583E493FAAE
:10140E00740193FBC3EF9BEE9A4008906F13E004B8
:10141E00F080D3ED75F003A42467F582E43422F551
:10142E0083C37401939FFFE4939EFEE4FCFD7BE86F
:10143E007A03F9F81204EDC8ECC8C9EDC9CAEECAB0
:10144E00CBEFCB906F13E0FF75F003A42469F58208
:10145E00E43422F583E493FDEF75F003A42466F5DE
:10146E0082E43422F583E493C39DFFE49400FEE40A
:10147E00FCFD1204EDECC0E0EDC0E0EEC0E0EFC00C
:10148E00E0906F13E0FF75F003A42464F582E4345A
:10149E0022F583E493FC740193FDEF75F003A4240D
:1014AE0067F582E43422F583C37401939DFFE493C0
:1014BE009CFEE4FCFDF8F9CAEECACBEFCBD0E0FF00
:1014CE00D0E0FED0E0FDD0E0FC120578EEC0E0EFFB
:1014DE00C0E0906F13E075F003A42469F582E43444
:1014EE0022F583E493FFE4FCFDFE7BE87A03F9F832
:0C14FE001204EDD0E02FFFD0E03EFE22F3
:10213700201175906F72E05407906F0AF0C39403F3
:102147004066E064076061D2117F01122F8FE4902F
:102157006F0AF07F017D127B03123059301706E5B5
:102167006860F980397F017D0E7B03123059301783
:1021770006E56860F980277F017D0A7B02123059E6
:10218700301706E56860F98015906F0AE004F0E003
:10219700B403C07F0112302E7F0A122F8F227F02D5
:0921A70012302E7F0A122F8F2244
:1012AE00301203021388E56864036009E568640B75
:1012BE0060030213EDD378D5E6954F18E6954E40B0
:1012CE000A906F11E4F0A304F0803BAF4FAE4E12C4
:1012DE0013EEEEC0E0EFC0E078D4E6FE08E6FF12B3
:1012EE0013EECCEECCCDEFCDD0E0FFD0E0FEC3EDD3
:1012FE009FFFEC9EFE906F11F0A3EFF04E700790E3
:10130E006F11F0A304F0D201E4906F0AF0906F1108
:10131E00E0FAA3E0FB7C007D0AFFCEEACE12043693
:10132E00906F0AE0240BF582E4346FF583EDF07CC8
:10133E00007D0ACFEBCFCEEACE120436906F11EEBF
:10134E00F0A3EFF0906F0AE004F0E0B405BF906FE9
:10135E000A7404F0906F0AE0FFF46015740B2FF519
:10136E0082E4346FF583E07008906F0AE014F08029
:10137E00E3EF04906F10F0D212227F1E122F8F7F98
:10138E00017D327B041230593017043016FA227F59
:10139E000A122F8F906F10E014906F0AF0906F0A60
:1013AE00E0240BF582E4346FF583E0700B7F017D52
:1013BE000B7B041230598016906F0AE0240BF582D5
:1013CE00E4346FF583E0FF7D0B7B0112305930174B
:1013DE00043016FA22906F0AE0FF14F0EF70BE226E
:10203400D2AF122E57122FB212000E122E8A123065
:102044009312300812000312229D122F167BFF7A7E
:102054002279271200C9122FFE122AAA50107BFFE0
:102064007A2279361200C97F0112302E800B7BFF51
:102074007A2279481200C9D211121FA0906EE7E0AB
:10208400FF122A38122CBC122784906EE8E0FEA3BB
:10209400E0FF12293B7BFF7A22795E1200C9C2124B
:1020A400C211301603122DCC1212AE906EDFE06016
:0720B400F112213780EC223C
:03000B00022313BA
:10231300C0E0C0F0C083C082C0D075D008C28CAF0B
:102323008CEFFEAD8AED255F78D7F6E55E3E18F6B5
:10233300F58C08E6F58AD28CD56309906EDEE0F55C
:1023430063122660D5621B906EDEE0F5620561E5DF
:102353006170020560E56145607007E568600375BB
:102363006805E5686404600F12182812259B121D86
:10237300A5122BB8121F03D0D0D082D083D0F0D0B7
:02238300E03246
:10293B00E4FCFDFB7AC079A8F81204ED7BE07A2E5B
:10294B00790078001228F7C374129FF55FE49EF5A7
:10295B005E906EDEE0F563F562E4F560F561E589A6
:10296B0054F04401F589758CFF758AFFC2B9D2A961
:03297B00D28C22D9
:0C2FCE00906EDEE0F562E4F560F5612233
:10278400E5C520E3FB75C50775C50FE5C530E4FB5A
:10279400AFC6EF75F004A4FFAEF0E5C5C41313543F
:1027A400037C002FF53CEC3EF53BE4F53AE53A2595
:1027B400E024C0F8A63B08A63CE53C2527F527E520
:1027C4003B3526F526053AE53AB40AE1E4F5392223
:10182800C0D075D008E5C520E3FBE4F5C575C5084B
:10183800F543754401E543640870030218FDE5C5E6
:1018480030E4FB85C62885C53DE5436407600EE5A1
:10185800C520E3FBE54304F5C54408F5C5E528754F
:10186800F004A4FFAEF0E53DC4131354037C002F2D
:10187800F546EC3EF545E54325E02429F8A645085C
:10188800A646906EDDE055446060AF28122AE3AFAB
:101898003D122AE3E543B406088545418546428062
:1018A80049E54364077043E53925E024C1F8C3E5F9
:1018B8002796F527E5261896F526E53925E024C06C
:1018C800F8A64508A646E5462527F527E545352621
:1018D800F526FEAF277C007D0A1204368E248F255C
:1018E8000539E539B40A03E4F5390543E54425E04B
:1018F800F54402183D300F1EE4A2C492E4A2C5923A
:10190800E5A29692E6A29792E72568C4F53EAF3E17
:0D191800122AE3853E40C294D294D0D02222
:10238500C0D075D008300F65906EE7E0FD7C0090F9
:102395006EF1E0FB24FFFFE434FFFE120422EF247C
:1023A50001FFE43EFEC3E51F9FF51FE51E9EF51EDA
:1023B5008B3FE53F6021E51EF583E51FF582E0C40F
:1023C50054F02568C4F0906EE7E0251FF51FE4354D
:1023D5001EF51E153F80DB906EE7E024FFFFE43419
:1023E500FFFEC3E51F9FF51FE51E9EF51ED0D022FB
:0D2FC100E4F576F577F578C219122A712231
:10259B00C0D075D008E5686057201954122F7C40C5
:1025AB004F906EE7E02404906F04F0906F04E060AE
:1025BB003F20133C122B848F7512002E0577E57785
:1025CB00700205767004E5766480701CF576F577FD
:1025DB000578E578B40C04D2198015122F69E578CB
:1025EB0020E005122A718008906F04E014F080BB84
:0325FB00D0D0221B
:102CBC00E4906FB0F0A3F0906FAC120650000000DF
:102CCC000074FF78D4F608F6E4906FB2F0F569F56D
:082CDC0068906FAB74FFF02259
:102E3D00C0D075D008756801AF68122EBAC2901255
:0A2E4D002FC17F0212302ED0D022D8
:102EEA00C0D0C291E5612401906FAAF0E4356090E8
:062EFA006FA9F0D0D02208
:102F0000C0D0C292E5612401906FAAF0E4356090D0
:062F10006FA9F0D0D022F1
:10116A00C0D075D008E4906F04F020C604E04401B2
:10117A00F020C707906F04E04402F0906FABE0FFE5
:10118A00906F04E0FE6F603BEE7025906FB8E0FF51
:10119A006005123036802C906FB7E0FF640360045C
:1011AA00EFB40405123036801A7F0112302E8013F4
:1011BA00906F04E030E0077F0112303680057F022D
:1011CA00123036906F04E0906FABF0300B1EA29491
:1011DA00300C01B34016C21A122FCE906EDBE0FE1D
:1011EA00A3E0FF122BE8122E3D0212AB20100302DD
:1011FA0012AB906EDAE0C4F8540FC868FF906ED94B
:10120A00E0C454F048FEC3E54D9FFDE54C9EFCE565
:10121A0042C4F8540FC868FFE541C454F048FED3ED
:10122A00EF9DEE9C4016D21A906FAC120650000049
:10123A000000E4906FB0F0122FCE8065C21A906F52
:10124A00ACE0F8A3E0F9A3E0FAA3E0FBE8C0E0E52C
:10125A0042C4F8540FC868FFE541C454F048FEC3BD
:10126A00EF954DFFEE954CFE3395E0FDFCD0E0F88E
:10127A00EB2FFFEA3EFEE93DFDE83CFC906FAC1225
:10128A000644906EF1E0FF906FB0E004F06F7011C9
:10129A00906EE2E0FEA3E0FF122BE8122E3D12232D
:0412AA0085D0D022F9
:101E5E00C0D075D008906FACE0F8A3E0F9A3E0FA1B
:101E6E00A3E0FBE8C0E0E542C4F8540FC868FFE504
:101E7E0041C454F048FEC3EF954DFFEE954CFE3332
:101E8E0095E0FDFCD0E0F8EB2FFFEA3EFEE93DFDCC
:101E9E00E83CFC906FAC120644300E387F007E009A
:101EAE007D007C00906FACE0F8A3E0F9A3E0FAA30C
:101EBE00E0FBD312060A401C906ED8E0FFD3E5611A
:101ECE009FE5609400400D122EEA756802AF68120D
:101EDE002EBA801E300D1B906EEDE0FEA3E0656104
:101EEE007003E5606E700B122EEA75680AAF681209
:051EFE002EBAD0D02235
:1021B000C0D075D008906FA9E0FEA3E06561700300
:1021C000E5606E7002D291300E3C906EE5E0FEA3A9
:1021D000E0FFC3E54F9FFFE54E9EFEC3E5259FE56B
:1021E000249E5007E4906FB1F0801B906F02E0FFD7
:1021F000906FB1E004F06F700D122F00756803AF9F
:1022000068122EBA801E300D1B906EEFE0FEA3E028
:1022100065617003E5606E700B122F0075680BAF7F
:0722200068122EBAD0D02293
:102DEA00C0D075D008906FA9E0FEA3E065617003BA
:0C2DFA00E5606E7004D291D292D0D0221D
:101DA500C0D075D008E5687003021E33E4F564758C
:101DB5006701E56464086065E56425E024F2F58261
:101DC500E4346EF583E0FEA3E08E65F566F47003FA
:101DD500E565F4603EE56955677015E56165667012
:101DE50004E56065657009E5674269AF64122820FE
:101DF500E5695567601DE5662401FFE43565FEEF7D
:101E050065617003EE6560700AE567F45269AF6459
:101E15001228B00564E56725E0F5678095C3E525DB
:101E250078D596E52418965005A62408A625E568D4
:101E350014601614601814601A24F96011146013E4
:101E4500240B701212116A800D121E5E8008122179
:091E5500B08003122DEAD0D02266
:102A3800CBEFCBEBFD7C007E3A7F98120436CDEBD2
:102A4800CD7C001204228E1A8F1B74002FF582EEA3
:102A58003434AF82F5188F197E347F008E1C8F1D99
:092A68008E1E8F1FD213C214222E
:102AE300201933C213051FE51FAC1E7002051E1407
:102AF300F5828C83EFF0E51F65197004E51E6518F8
:102B03007006751E34751F00E51F651D7004E51EF4
:072B1300651C7002D21422C0
:102B8400C214051DE51DAE1C7002051C14F5828ED1
:102B940083E0FFE51D65197004E51C651870067572
:102BA4001C34751D00E51F651D7004E51E651C7051
:042BB40002D2132214
:102BE800C3E51F9FF51DE51E9EF51CC3E51D94005A
:102BF800E51C9434400BD3E51D9519E51C95184048
:0E2C08000CE51B251DF51DE51A351CF51C22DB
:101C0C002573202562752025627520257520257584
:101C1C0020257520257520256320256275202563D8
:101C2C002025632025630D0A00632069676E20253B
:101C3C007520257520257520257520257520257581
:101C4C002025752025750D0A006320786D69742098
:101C5C00257520256275202562750D0A00632067A5
:101C6C007073202562750D0A00696E6465780065D5
:101C7C0072617365006F6666006F6E002A5645527E
:101C8C0053494F4E3A20522D4441532056332E3354
:101C9C000D0A006321006320726461730063206984
:101CAC00676E006320786D69740063206770730041
:101CBC00633F0063006320006770732000726573DC
:101CCC006574002A453A20756E6B6E6F776E2063D3
:051CDC006D640D0A001B
:08000300E4F57EC216C21522CD
:1008F900906F0AEBF0A3EAF0A3E9F0300B13300C88
:1009090008906F277401F0800D906F277402F080B2
:1009190005E4906F27F0906F0AE0FBA3E0FAA3E0EB
:10092900F91203BA643F60030209DF906F0DE0F921
:10093900A3E0FAA3E0906F32C9F0A3EAF0A3E9F0CB
:10094900906EDEE0906F35F0906EDDE0906F36F0DE
:10095900906ED9E0FFA3E0906F37CFF0A3EFF0904E
:100969006EE5E0FFA3E0906F39CFF0A3EFF0906E52
:10097900EDE0FFA3E0906F3BCFF0A3EFF0906EEFB7
:10098900E0FFA3E0906F3DCFF0A3EFF0300F047FBD
:100999003180027F30906F3FEFF0906F27E0906FCA
:1009A90040F03010047F3180027F30906F41EFF0CA
:1009B900300E047F3180027F30906F42EFF0300DAE
:1009C900047F3180027F30906F43EFF07BFF7A1C08
:1009D900790C1200C922906F0AE0FBA3E0FAA3E0A8
:1009E900F91203BAFF122F2C500C906F0BE475F01B
:1009F900011204C180E0E4906F26F0906F0AE0FBD9
:100A0900A3E0FAA3E0F9121618906F26E025E02476
:100A190010F582E4346FF583EEF0A3EFF0906F0ADE
:100A2900E0FBA3E475F0011204D7A9F0FA1203BAA6
:100A3900FF122F2C50E7906F26E004F0E0B40BBBB7
:100A4900906F11E0906EDEF0906F13E0906EDDF024
:100A5900906F14E0FFA3E0906ED9CFF0A3EFF09070
:100A69006F16E0FFA3E0906EE5CFF0A3EFF0906F73
:100A790018E0FFA3E0906EEDCFF0A3EFF0906F1AAE
:100A8900E0FFA3E0906EEFCFF0A3EFF0906F1CE0D2
:100A9900FEA3E0FFEE4F24FF920FA3E0FEA3E0FFC9
:100AA900EE4F24FF920BEF64014E7003D38001C314
:100AB900920C906F20E0FEA3E0FFEE4F24FF92100E
:100AC900A3E0FEA3E0FFEE4F24FF920EA3E0FEA3F6
:090AD900E0FFEE4F24FF920D2214
:10172600906F0AEBF0A3EAF0A3E9F01203BA643F64
:1017360060030217BD7BFF7A1C7935906EF2E0FFDD
:10174600A3E0906F32CFF0A3EFF0906EF4E0FFA32A
:10175600E0906F34CFF0A3EFF0906EF6E0FFA3E0D9
:10176600906F36CFF0A3EFF0906EF8E0FFA3E09015
:101776006F38CFF0A3EFF0906EFAE0FFA3E0906F22
:101786003ACFF0A3EFF0906EFCE0FFA3E0906F3C41
:10179600CFF0A3EFF0906EFEE0FFA3E0906F3ECF98
:1017A600F0A3EFF0906F00E0FFA3E0906F40CFF062
:1017B600A3EFF01200C922906F0AE0FBA3E0FAA3A0
:1017C600E0F91203BAFF122F2C500C906F0BE47540
:1017D600F0011204C180E0E4906F0DF0906F0AE012
:1017E600FBA3E0FAA3E0F9121618906F0DE025E0CE
:1017F60024F2F582E4346EF583EEF0A3EFF0906FF9
:101806000AE0FBA3E475F0011204D7A9F0FA12036B
:10181600BAFF122F2C50E7906F0DE004F0E0B408E9
:02182600BB22E3
:101CE100906F0AEBF0A3EAF0A3E9F01203BAB43F54
:101CF100297BFF7A1C7955906EE0E0FFA3E0906F9D
:101D010032CFF0A3EFF0906EEAE0906F34F0906F75
:101D110003E0906F35F01200C922906F0AE0FBA337
:101D2100E0FAA3E0F91203BAFF122F2C500C906FC6
:101D31000BE475F0011204C180E0E4906F13F090A0
:101D41006F0AE0FBA3E0FAA3E0F9121618906F13F3
:101D5100E025E0240DF582E4346FF583EEF0A3EF86
:101D6100F0906F0AE0FBA3E475F0011204D7A9F02B
:101D7100FA1203BAFF122F2C50E7906F13E004F010
:101D8100E0B403BB906F0DE0FFA3E0906EE0CFF0F5
:101D9100A3EFF0906F10E0906EEAF0906F12E09078
:041DA1006F03F022BA
:1025FE00906F0AEBF0A3EAF0A3E9F0906F0AE0FB0C
:10260E00A3E0FAA3E0F91203BAB43F127BFF7A1CDF
:10261E007969906EDFE0906F32F01200C922906FF0
:10262E000AE0FBA3E0FAA3E0F91203BAFF122F2C83
:10263E00500C906F0BE475F0011204C180E0906FA6
:10264E000AE0FBA3E0FAA3E0F9121618906EDFEF92
:02265E00F02268
:1006F9007B017A6E799A7D20122E06906F0DEBF0B0
:10070900A3EAF0A3E9F04A70047F0180027F009018
:100719006F1AEFF0605F7B017A6E7999121618C82B
:10072900ECC8C9EDC9CAEECACBEFCB906EEBE0FEBF
:10073900A3E0FFE4FCFD1204EDC8ECC8C9EDC9CA89
:10074900EECACBEFCB906EDBE0FEA3E0FFE4FCFD4D
:10075900EB2FFFEA3EFEED39FDEC38FC906F1012ED
:100769000644906EEBE0FEA3E0FFE4FCFD906F14FD
:1007790012064480767B017A6E7999121618C8ECB4
:10078900C8C9EDC9CAEECACBEFCB906EE7E0FFE46A
:10079900FCFDFE1204EDC8ECC8C9EDC9CAEECACB0E
:1007A900EFCB906EDBE0FEA3E0FFE4FCFDEB2FFF57
:1007B900EA3EFEED39FDEC38FC906F1012064490CC
:1007C9006F0DE0FBA3E0FAA3E0F9121618C8ECC814
:1007D900C9EDC9CAEECACBEFCB906EE7E0FFE4FCE6
:1007E900FDFE1204ED906F14120644906F10E0FCA8
:1007F900A3E0FDA3E0FEA3E0FF780F1206318F7896
:10080900906F10E0FCA3E0FDA3E0FEA3E0FFEE542F
:100819007FFEE48E768F77122F69906F1AE0600958
:10082900E4906F18F0A3F0800B120026906F18EE79
:10083900F0A3EFF0E4906F0AF0A3F0906F0AE0FEE6
:10084900A3E0FFE4FCFD906F14E0F8A3E0F9A3E056
:10085900FAA3E0FBC3120620606C122FDA906F0C2A
:10086900EFF0906F1AE06014906F0CE0FF906F1931
:10087900E02FF0906F18E03400F08018906F18E0C6
:10088900FEA3E0FF906F0CE0FD1220BB906F18EE05
:10089900F0A3EFF0906F0CE0FF1230260577E577B3
:1008A900700205767004E57664807009F576F5774F
:1008B9000578122F69906F0BE004F07006906F0AAB
:1008C900E004F0020844906F1AE07013906F18E08A
:1008D900FEA3E0FF12304C906F18EEF0A3EFF090FA
:1008E9006F18E0FF123026906F19E0FF12302622B0
:102F4100D3EF648094B95007EF24D0FEFF8004EFE3
:042F510024A9FF228E
:10192500906F0AEBF0A3EAF0A3E9F0906F1174FF52
:10193500F0A3741CF0A37475F0A3E4F0A37405F090
:10194500122534EF7003122868906F1174FFF0A30D
:10195500741CF0A3747BF0A3E4F0A37405F0906FFE
:101965000AE0FBA3E0FAA3E0F9122534EF700412B4
:101975002E7122906F1174FFF0A3741CF0A3748173
:10198500F0A3E4F0A37403F0906F0AE0FBA3E0FA80
:10199500A3E0F9122534EF7003C21522906F11747C
:1019A500FFF0A3741CF0A37485F0A3E4F0A3740204
:1019B500F0906F0AE0FBA3E0FAA3E0F9122534EFFB
:1019C5007003D21522906F0AE0FBA3E0FAA3E0F9B9
:1019D5001203BAFF122C935043906F0AE0FBA3E069
:1019E500FAA3E0F99000011203D3FF122F41CDEFC6
:1019F500CD906F0AE0FBA3E0FAA3E0F91203BAFF6A
:101A0500122F41EFC454F02DFF906F0DF0122EA24E
:0D1A1500906F0BE475F0021204C180A9224D
:04308300122D2A22BE
:0A2FFE007BFF7A1C79881200C922BB
:100AE200906F1174FFF0A3741CF0A3749FF0A3E441
:100AF200F0A37402F07B017A6E7998122534EF70BC
:100B020004120CB422906F1174FFF0A3741CF0A3B2
:100B120074A2F0A3E4F0A37406F07B017A6E7998D4
:100B2200122534EF7018906F0D74FFF0A3741CF04F
:100B3200A374A2F07B017A6E799E1208F922906F5B
:100B42001174FFF0A3741CF0A374A9F0A3E4F0A342
:100B52007405F07B017A6E7998122534EF700A7B66
:100B6200017A6E799D12172622906F1174FFF0A3FD
:100B7200741CF0A374AFF0A3E4F0A37406F07B013D
:100B82007A6E7998122534EF700A7B017A6E799E1B
:100B9200121CE122906F1174FFF0A3741CF0A37475
:100BA200B6F0A3E4F0A37405F07B017A6E79981293
:100BB2002534EF700A7B017A6E799D1225FE229010
:100BC2006F1174FFF0A3741CF0A374BCF0A3E4F0E3
:100BD200A37402F07B017A6E7998122534EF7018B3
:100BE200906F0D74FFF0A3741CF0A374BFF07B012F
:100BF2007A6E79991208F922906F1174FFF0A3743A
:100C02001CF0A374C1F0A3E4F0A37402F07B017A98
:100C12006E7998122534EF7018906F0D74FFF0A35F
:100C2200741CF0A374BFF07B017A6E79991208F9F3
:100C320022906E98E0B464041206F922906F117447
:100C4200FFF0A3741CF0A374C4F0A3E4F0A3740433
:100C5200F07B017A6E7998122534EF700A7B017A63
:100C62006E799C12192522906F1174FFF0A3741CE7
:100C7200F0A374C9F0A3E4F0A37405F07B017A6ECB
:100C82007998122534EF700412308322906E98E026
:100C9200B46904121A2222906E98E0B47604122FDC
:100CA200FE22906E98E060097BFF7A1C79CF1200D9
:020CB200C92255
:102DCC0010160280107568047F0112302E7F1E12BF
:0E2DDC002F8F120AE23015E81226C280E32281
:102B1A00C0D0EF20E72CEF640A6027EF640D601144
:102B2A007498257EF582E4346EF583EFF0057E8095
:102B3A00117498257EF582E4346EF583E4F0D2169A
:052B4A00F57ED0D02251
:1023F5002A4D4553534147453A2053746F72696ED0
:102405006720706172616D657465727320696E20F5
:10241500464C4153480D0A002A4D45535341474503
:102425003A2046696E69736865642073746F7269D2
:102435006E670D0A00000001C001C802000C001BF8
:1024450001000019003C03FFFFFFFFFFFFFFFFFF37
:0C245500FFFFFFFFFFFFFF00000A010077
:0A300800757C24757D3A120FEC224E
:100FEC0090243AE49324FF920BA3E49324FF920CF5
:100FFC00A3E49324FF9210A3E493906EDDF090246D
:10100C003EE49324FF920FE4906EE7F07F80EF6054
:10101C0014906EDDE05F6007906EE7E02402F0EF65
:10102C00C313FF80E9300F06906EE7E004F09024C4
:10103C003FE493906EDEF0902440E493906EE4F0E5
:10104C00902441E493FF740193906ED9CFF0A3EFF9
:10105C00F0902443E493FF740193906EE5CFF0A3DA
:10106C00EFF0906EDEE0FBFD7C007E037FE8120467
:10107C0036906EE8EEF0A3EFF0906EE7E0FA8BF0AE
:10108C00A4FF906EEBE5F0F0A3EFF0EB1313543FDD
:10109C00906EF1F0FB906F02F0902445E49324FFE6
:1010AC00920EA3E49324FF920DA3E493FF74019397
:1010BC00906EEDCFF0A3EFF0902449E493FF740110
:1010CC0093906EEFCFF0A3EFF090244BE493906EDF
:1010DC00D8F0906EE4E0FF7E00906EEBE0FCA3E0B5
:1010EC00FD120422906EDBEEF0A3EFF0EBFF7E001E
:1010FC00EAFD7C00120422E02F906EE3F0906EDB90
:10110C00E03E906EE2F0E4FFEF25E0244CF582E443
:10111C003424F583E493FC740193FDEF25E024F271
:10112C00F582E4346EF583ECF0A3EDF00FEFB40828
:10113C00D790245CE493FF740193906EE0CFF0A3FE
:10114C00EFF090245EE493906EEAF090245FE493C9
:0E115C00906F03F0902460E493906EDFF02219
:100CB400A20BE433857D82857C83F0A20CE433A30C
:100CC400F0A210E433857D82857C83A3A3F0906E2B
:100CD400DDE0857D82857C83A3A3A3F0A20FE433AA
:100CE400FFE57D2404F582E4357CF583EFF0906E16
:100CF400DEE0FFE57D2405F582E4357CF583EFF045
:100D0400906EE4E0FFE57D2406F582E4357CF5830E
:100D1400EFF0906ED9E0FEA3E0FFE57D2407F582B5
:100D2400E4357CF583EEF0A3EFF0906EE5E0FEA3EE
:100D3400E0FFE57D2409F582E4357CF583EEF0A33C
:100D4400EFF0A20EE433FFE57D240BF582E4357C5D
:100D5400F583EFF0A20DE433FFE57D240CF582E486
:100D6400357CF583EFF0906EEDE0FEA3E0FFE57DCA
:100D7400240DF582E4357CF583EEF0A3EFF0906E5C
:100D8400EFE0FEA3E0FFE57D240FF582E4357CF57A
:100D940083EEF0A3EFF0906ED8E0FFE57D2411F52B
:100DA40082E4357CF583EFF0E4906F0AF0906F0AEB
:100DB400E0FF6408603BEF25E024F2F582E4346E42
:100DC400F583E0FEA3E0FFE57D2412F582E4357CA3
:100DD400F583C083C082906F0AE0D082D08375F01F
:100DE40002120681EEF0A3EFF0906F0AE004F080A7
:100DF400BC906EE0E0FEA3E0FFE57D2422F582E4F2
:100E0400357CF583EEF0A3EFF0906EEAE0FFE57D2C
:100E14002424F582E4357CF583EFF0906F03E0FF42
:100E2400E57D2425F582E4357CF583EFF0906EDFD3
:100E3400E0FFE57D2426F582E4357CF583EFF07B45
:100E4400FF7A2379F51200C9122B4F7BFF7A24799C
:050E54001D1200C9227F
:101FA000E5C520E3FB75C50675C50EE5C530E4FB48
:101FB000AFC6EF75F004A4FFAEF0E5C5C41313542B
:101FC000037C002FF54DEC3EF54CE5C520E3FB7599
:101FD000C50775C50FE5C530E4FBAFC6EF75F00466
:101FE000A4FFAEF0E5C5C4131354037C002FF54ADB
:101FF000EC3EF549F54E854A4FD21AE4F547F548CF
:10200000FFEF25E02479F582E4346FF583E54CF0A9
:10201000A3E54DF0E54D2548F548E54C3547F54736
:102020000FEFB410DCE4F54BE5482401F54DE43541
:0420300047F54C2202
:10266000301A5EE5482401F54DE43547F54CE54B5D
:1026700025E02479F582E4346FF583E0FEA3E0FFE2
:10268000C3E5489FF548E5479EF547E54B25E0241F
:1026900079F582E4346FF583E541F0A3E542F0E596
:1026A000422548F548E5413547F547054BE54BB42C
:1026B0001003E4F54B85494E854A4F85244985250D
:0226C0004A22AC
:102E5700D21B43878075985AE589540F4420F5891A
:0A2E6700758DFFD28ED2BCD2AC22D2
:03002300022C416B
:102C4100C0E0C0F0C083C082C0D075D010309807FA
:102C5100AF99C298122B1A309904C299D21BD0D0C5
:092C6100D082D083D0F0D0E03223
:08302600301BFDC21B8F992233
:07303E00CEEFCE1230262276
:102C6A00E5C520E3FB8FC5EF4408F5C5E5C530E4AB
:102C7A00FBAFC6EF75F004A4FFAEF0E5C5C41313AD
:092C8A005403FDE5F0EF4DFF22BB
:102D2A00E4F5A8F5E8F5B8F5F875780FE578A2E0C6
:102D3A0092B5A2E192B3A2E292B4A2E392B202FFE6
:022D4A00FE2267
:102F6900E578A2E092B5A2E192B3A2E292B4A2E31B
:032F790092B222EF
:0C2FDA00E5764480857782F583E0FF22D5
:10002E0090D3557499F090ACAA7466F090D3557431
:10003E0090F0E575F5F0E576D2E7F583E577F58294
:0D004E00E5F0F0E0A2E730F701B340F72243
:102A7100E578A2E092B5A2E192B3A2E292B4A2E318
:102A810092B290D3557499F090ACAA7466F090D339
:102A9100557480F090D3557499F090ACAA7466F097
:092AA1009080007414F0D21C2294
:102F7C00301C0D908000E020E703D38001C3921C2D
:032F8C00A21C2262
:102B4F0075780C122A71122F7C40FB75780D122F9D
:102B5F0069E4F576F577857782857683E0F57512EA
:102B6F00002E0577E57770020576E5777004E57638
:052B7F00648070E222F9
:03309300C21C223A
:03005B000224611B
:10246100C0E0C0D0C2CC742D25C9F5C930175815AC
:1024710050E5507052E55670128552FCC2C0F551BC
:10248100755601E55425E0F550803CE55664017030
:102491002375FCFFD2C00551E5516553700E30180C
:1024A10007F556855550801FC217801B755602755A
:1024B10050028013E556B4020E8552FCC2C0755617
:0C24C10001E55425E0F550D0D0D0E03209
:102E8A0075FCFFD2C075FE0B75528075EA0DC2FC47
:082E9A00D2EC75550AC21722A3
:102CE400C217A202921875FCFFD2C08F53E4F556A6
:102CF400CEEDCE8EFECEEBCE8E54855550EF6002D7
:032D0400D21722C1
:06305300D202122CE4225F
:06305900C202122CE42269
:08302E007D0B7B0112305322DF
:083036007D327B0412305322AD
:102F8F00C21775FCFFD2C08F55E4F556855550D248
:022F9F001722F7
:10150A00413A253475202534752025347520253433
:10151A007520253475202534752025347520253409
:10152A007520443A25303262782043433A256325B0
:10153A00632042573A25630D0A002A4D3A20615F1B
:10154A007374203D2025750D0A002A4D3A20612822
:10155A003029203D2025750D0A002A573A20615F5F
:10156A0073743D25752C2061303D25752028672D23
:10157A0073772064697361626C6564290D0A002AB5
:10158A004D3A2070283029203D2025750D0A002A61
:10159A00573A20502072616E6765205B25752C25AD
:1015AA00755D0D0A002A573A204257206572726FFC
:1015BA0072202842572064697361626C6564290D40
:1015CA000A002A573A206E6F2069676E20256264E6
:1015DA000D0A002A573A206E6F20786D69740D0A39
:1015EA00002A573A206E6F206770730D0A002A5737
:1015FA003A2064726F677565206572720D0A002A57
:0E160A00573A206D61696E206572720D0A00FC
:07304500EF60031F80FA2277
:101A22001016028003021B19E4A2C492E0A2C5921E
:101A3200E1A29692E2A29792E3F57BE4FF122C6A6E
:101A4200EFC0E0EEC0E07F01122C6AEFC0E0EEC012
:101A5200E07F02122C6AEFC0E0EEC0E07F03122C9E
:101A62006AEFC0E0EEC0E07F04122C6AEFC0E0EE45
:101A7200C0E07F05122C6AEFC0E0EEC0E07F0612E4
:101A82002C6AEFC0E0EEC0E07F07122C6A906F4034
:101A9200EEF0A3EFF0906F3ED0E0F0A3D0E0F09034
:101AA2006F3CD0E0F0A3D0E0F0906F3AD0E0F0A32A
:101AB200D0E0F0906F38D0E0F0A3D0E0F0906F3635
:101AC200D0E0F0A3D0E0F0906F34D0E0F0A3D0E00B
:101AD200F0906F32D0E0F0A3D0E0F07BFF7A15797E
:101AE2000A906F42E57BF030C6047F6380027F6F0D
:101AF200906F43EFF030C7047F6380027F6F906F77
:101B020044EFF03094047F6F80027F63906F45EF63
:081B1200F01200C9021A2222A0
:102DAD00A2029293E4F579F57A7F78123045057A8F
:0F2DBD00E57A70020579E57A640A457970EB22B0
:100E5900E4906F0FF0906F0AF0A3F0906F0EF0D24C
:100E690002122DAD7F06122C6A906F0BE02FF090C5
:100E79006F0AE03EF0C202122DAD906F0EE004F051
:100E8900E0B420DB906F0AE0FEA3E0FF7C007D2048
:100E990012048B906F0AEEF0A3EFF07BFF7A1579BD
:100EA90044906F32EEF0A3EFF01200C9E4906F0C9A
:100EB900F0A3F0A3F07F06122C6A906F0DE02FF0DB
:100EC900906F0CE03EF0906F0EE004F0E0B420E586
:100ED900906F0CE0FEA3E0FF7C007D2012048B9054
:100EE9006F0CEEF0A3EFF07BFF7A157954906F3217
:100EF900EEF0A3EFF01200C9906F0CE0FEA3E0FF43
:100F0900906F0AE0FCA3E0FDC39FFFEC9EFEC3EFD8
:100F1900942DEE64809480502D7BFF7A157964902E
:100F29006F32ECF0A3EDF0906F0CE0FFA3E0906F4F
:100F390034CFF0A3EFF01200C97F06123036C21089
:100F4900906F0F7406F0E4906F0AF0A3F0906F0EA3
:100F5900F07F07122C6A906F0BE02FF0906F0AE078
:100F69003EF0906F0EE004F0E0B420E5906F0AE0E7
:100F7900FEA3E0FF7C007D2012048B906F0AEEF047
:100F8900A3EFF07BFF7A157989906F32EEF0A3EF2A
:100F9900F01200C9906F0AE0FEA3E0FFC3947DEE52
:100FA90064809482400BD3EF94DBEE648094834099
:100FB9002C7BFF7A157999906F32EEF0A3EFF0A3AD
:100FC9007402F0A3747DF0A37403F0A374DBF01230
:100FD90000C97F05123036906F0F7405F0906F0FBE
:030FE900E0FF2204
:101B1A00E4906F0AF0300B1EA294300C01B3401609
:101B2A007BFF7A1579AF1200C97F03123036C20BD8
:101B3A00906F0A7403F0E4906F0BF0906F0BE0FF64
:101B4A006408606AEF25E024F2F582E4346EF583D6
:101B5A00E0FCA3E0F47002ECF4604B122FE6401FA5
:101B6A007F041230367BFF7A1579CC906F0BE00434
:101B7A00906F32F01200C9906F0A7404F0802790B7
:101B8A006F0BE0FF1227D4401D7F041230367BFF13
:101B9A007A1579CC906F0BE004906F32F01200C97D
:101BAA00906F0A7404F0906F0BE004F0808D906ED1
:101BBA00E0E07002A3E06020123065401B7F04124F
:101BCA0030367BFF7A1579DD1200C9E4906EE0F0B9
:101BDA00A3F0906F0A7404F0906EDFE0601E12307A
:101BEA005F40197F041230367BFF7A1579EB1200B9
:101BFA00C9E4906EDFF0906F0A7404F0906F0AE007
:021C0A00FF22B7
:102AAA00D201121B1A906FB7EFF06002C201120E28
:102ABA0059906FB8EFF06002C20120C60B7BFF7A13
:102ACA001579F81200C9C20120C70B7BFF7A167963
:092ADA00091200C9C201A2012287
:10000E00E4FF74B32FF582E4346FF58374FFF00FC1
:05001E00EFB404EE2226
:0C2FE600EFC31325E02441FF122E22222D
:1027D400906F0CEFF0E0FFC31325E02441FF7B0171
:1027E4007A6F790E906F147401F012297E906F0D38
:1027F400EFF0906F0CE054012402FF74017E00C8D6
:10280400EFC8088005C333CE33CED8F9FF906F0EDE
:0C281400E0FDE4EF5D6003D38001C3220F
:10282000CEEFCEEEC313FF24B3F582E4346FF5830D
:10283000C083C082E0FDEE5401FC7401C8ECC808FE
:102840008002C333D8FCF45DD082D083F0EF25E062
:102850002440FFEEC31324B3F582E4346FAD82FC51
:082860007B01D2011229FD22C7
:1028B000CEEFCEEEC313FF24B3F582E4346FF5837D
:1028C000C083C082E0FDEE5401FC7401C8ECC8086E
:1028D0008002C333D8FC4DD082D083F0EF25E024B2
:1028E00040FFEEC31324B3F582E4346FAD82FC7B6A
:0728F00001D2011229FD22B3
:102F1600E4F57FFF746C2FF582E4346FF583E4F0FB
:062F26000FEFB40DEF22D5
:06305F007F50122E222218
:102EA200906F0EEFF07F507C6F7D0E7B01D201128E
:082EB20029FD906F0FEFF022E3
:1026C2007F537B017A6F790B906F147401F012299A
:1026D2007E906F0AEFF0A3E0D3941040037410F0E1
:1026E200906F0BE0FE603A7F517B017A6F7999908F
:1026F2006F14F012297E906F0AEFF0E4F0906F0BE6
:10270200E0FF906F0AE0FE6F601774992EF582E485
:10271200346FF583E0FF123026906F0AE004F080F8
:02272200DC22B7
:10286800E4906F0EF07F577B017A6F7999906F141F
:102878007410F012297E906F0FEFF0E4F0906F0F54
:10288800E0FF6410601774992FF582E4346FF583C4
:10289800E0FF12303E906F0FE004F080E0906F0E82
:0828A800E004F0E0B408BE22D8
:102E7100906F0E7442F07F567C6F7D0E7B01D20104
:092E81001229FD906F0FEFF02201
:102EBA00906F05EFF07F547C6F7D057B01C2011294
:082ECA0029FD906F06EFF022D4
:102BB800C0D075D008906EDFE06022057F906EDE91
:102BC800E0657F7018F57F7F557B017A6F79669095
:102BD8006F14740DF012297E906F04EFF0D0D0229C
:10229D00D21DE4F557F558F559906EDEE0FF75F057
:1022AD000A84755C00F55DEFC313755A00F55B90FC
:1022BD006EE0E0FEA3E0FF4E604B906F577404F0AC
:1022CD00E4A3F0FCFDF8F9CAEECACBEFCBFF7EC05C
:1022DD007DA81228F77B107A00790078001228F774
:1022ED00EF14906F59F0906F03E075F080A4FF909C
:1022FD006EEAE02F906F5AF07F607C6F7D577B0404
:06230D00D2011229FD229D
:063065007F60122E222202
:1024CD00C0E0A3E558F0A3E559F0A3E52AF0A3E594
:1024DD002CF0A3E52EF0A3E530F0A3E532F0A3E553
:1024ED0034F0A3E536F0A3E538F0A375F000E52947
:1024FD0042F0E52B232342F0E52DC442F0E52FC435
:10250D00232345F0F0A375F000E53142F0E53323C8
:10251D002342F0E535C442F0E537C4232345F0F0FE
:07252D00A3E540F0D0E0221D
:101F0300C0D075D008906EE0E07002A3E0700302C9
:101F13001F9D301D09E5686005E4F557C21DE557AF
:101F2300FB7A00AC5CAD5DFFCEEACE120436ED4C1D
:101F3300705C906EDFE0601DAC5AAD5BCFEBCFCE33
:101F4300EACE120436ED4C700C906F04741CF0A3AF
:101F53007402F0800A906F04740FF0A37401F09080
:101F63006F04E0906F57F0906F05E0906F58F01298
:101F730024CD7F607C6F7D57906F04E0FBC201121C
:101F830029FDE56860080559E559700205580557AC
:0D1F9300906EDEE065577002F557D0D02249
:102D6D000000CC01D8011400F0013C002800E40162
:102D7D00A0016C007800B40150009C018801440052
:050026007EFF7FFF22B8
:1020BB00CBEFCBCAEECAC9EDC9E9540FFFEAEB6F00
:1020CB00540F25E0FFE433FE746D2FF582EE342DB3
:1020DB00F583EAC4F854F0C868FEEBC4540F48FF0C
:1020EB00EE540FFEE4936EFA7401936FFBCFE9CFBE
:1020FB00EFC4540F540FFFEAEF6B540F25E0FFE4CE
:10210B0033FE746D2FF582EE342DF583EAC4F8544B
:10211B00F0C868FEEBC4540F48FFEE540FFEE49377
:0C212B006EFA7401936FFBCEEACEFF2227
:07304C00EEF4FEEFF4FF2299
:10272400FF3087FF3012FF301CFF2D4CFF306BFF52
:102734002D07FF3071FF308BFF2ED2FF3077FF2D36
:102744008DFF2F55FF308FFF3096FF3097FF309865
:10275400FF3099FF309AFF309BFF309CFF309DFF84
:10276400309EFF309FFF30A0FF30A1FF30A2FF302A
:102774007DFF307DFF307DFF307DFF307DFF307D7C
:0F2FB200D296D29775D8C575DBECD2BDD2AD22C1
:102E2200E4F56F8F6DD21ED2DDFF122C16EF6418FF
:0B2E32006004EFB44003D38001C32212
:1029FD00906F10ECF0A3EDF08C838D827880EBFE60
:102A0D006006E0F6A308DEFA8B6F8F6DD21ED2DD65
:102A1D0030010DCFEBCF122C16906F12EFF0800519
:0B2A2D00E4906F12F0906F12E0FF22A7
:10297E00906F11EBF0A3EAF0A3E9F0CEEFCEA3E057
:10298E00FFF56F8E6DD21ED2DD122C16E4FE906F07
:10299E0014E06E601D74802EF8E6FD906F11E0FB62
:1029AE00A3E0FAA3E0F98E82758300ED1204000E07
:0329BE0080DC2298
:102C1600CEEFCEE4F56AEE2402FDE433FCE56A6D00
:102C26007001EC6010756BDDD56BFD201E03AF6E79
:0B2C360022056A80E175D8D57F0022DE
:0430870075D8D52201
:0A301200856DDA75D8C5E4F56C226F
:0A301C00856DDA75D8C5E4F56C2265
:102D4C00C0D075D010E56F700775D8D5C21E800E37
:102D5C00AF6C056C74802FF8E6F5DA75D8C5D0D059
:012D6C002244
:06306B0075D8D5C21E223B
:102D0700C0D075D010E56C656F700775D8D5C21E39
:102D1700800EAF6C056C74802FF8E6F5DA75D8C5B0
:032D2700D0D022E7
:0630710075D8D5C21E2235
:04308B0075D8E522ED
:102ED200E56F14600A04700C75D8D5C21E8008759F
:082EE200D8C1800375D8C52298
:0630770075D8D5C21E222F
:102D8D00C0D075D0107480256CF8A6DAE56F1405E7
:102D9D006C656C700575D8C1800375D8C5D0D0220F
:102F5500C0D075D0107480256CF8A6DA75D8D5C2A6
:042F65001ED0D02288
:04308F0075D8D522F9
:013096002217
:013097002216
:013098002215
:013099002214
:01309A002213
:01309B002212
:01309C002211
:01309D002210
:01309E00220F
:01309F00220E
:0130A000220D
:0130A100220C
:0130A200220B
:06307D0075D8D5C21E2229
:03002B000229C1E6
:1029C100C0E0C0F0C083C082C0D075D01085D96E80
:1029D100E5D9131313541F75F003A42424F582E4DD
:1029E1003427F583E493740193FA740293F9120680
:0C29F1008DD0D0D082D083D0F0D0E03266
:03000000022FF2DA
:0C2FF200787FE4F6D8FD7581D70220340A
:1003BA00BB010689828A83E0225002E722BBFE0241
:0903CA00E32289828A83E4932274
:1003D300BB010CE58229F582E5833AF583E02250DF
:1003E30006E92582F8E622BBFE06E92582F8E22229
:0D03F300E58229F582E5833AF583E4932243
:10040000F8BB010DE58229F582E5833AF583E8F032
:10041000225006E92582C8F622BBFE05E92582C8DE
:02042000F222C6
:10042200EFF88DF0A4FFEDC5F0CEA42EFEEC88F01F
:04043200A42EFE22D4
:10043600BC000BBE0029EF8DF084FFADF022E4CCAA
:10044600F875F008EF2FFFEE33FEEC33FCEE9DEC73
:10045600984005FCEE9DFE0FD5F0E9E4CEFD22EDB9
:10046600F8F5F0EE8420D21CFEADF075F008EF2F03
:10047600FFED33FD4007985006D5F0F222C398FDF4
:050486000FD5F0EA2291
:10048B00C2D5EC30E709B2D5E4C39DFDE49CFCEE8C
:10049B0030E715B2D5E4C39FFFE49EFE120436C3CA
:1004AB00E49DFDE49CFC800312043630D507C3E4C5
:0604BB009FFFE49EFE22FB
:1004C100C5F0F8A3E028F0C5F0F8E58215827002C6
:0604D1001583E038F02263
:1004D700A3F8E0C5F025F0F0E582158270021583D8
:0604E700E0C838F0E82235
:1004ED00E88FF0A4CC8BF0A42CFCE98EF0A42CFCAE
:1004FD008AF0EDA42CFCEA8EF0A4CDA8F08BF0A42C
:10050D002DCC3825F0FDE98FF0A42CCD35F0FCEB8A
:10051D008EF0A4FEA9F0EB8FF0A4CFC5F02ECD394F
:0F052D00FEE43CFCEAA42DCE35F0FDE43CFC22BC
:10053C0075F008758200EF2FFFEE33FECD33CDCC76
:10054C0033CCC58233C5829BED9AEC99E5829840F9
:10055C000CF582EE9BFEED9AFDEC99FC0FD5F0D6D6
:10056C00E4CEFBE4CDFAE4CCF9A88222B800C1B900
:10057C000059BA002DEC8BF084CFCECDFCE5F0CB3E
:10058C00F97818EF2FFFEE33FEED33FDEC33FCEB77
:10059C0033FB10D703994004EB99FB0FD8E5E4F932
:1005AC00FA227818EF2FFFEE33FEED33FDEC33FC1F
:1005BC00C933C910D7059BE99A4007EC9BFCE99A13
:1005CC00F90FD8E0E4C9FAE4CCFB2275F010EF2F58
:1005DC00FFEE33FEED33FDCC33CCC833C810D70758
:1005EC009BEC9AE899400AED9BFDEC9AFCE899F893
:0E05FC000FD5F0DAE4CDFBE4CCFAE4C8F92226
:1028F700C2D5E830E70FB2D5E4C39BFBE49AFAE40C
:1029070099F9E498F8EC30E717B2D512292D12059A
:1029170078E4C39BFBE49AFAE499F9E498F8800316
:1029270012057830D50DE4C39FFFE49EFEE49DFDBC
:04293700E49CFC22FE
:10060A00EB9FF5F0EA9E42F0E99D42F0EC6480C867
:06061A0064809845F02207
:10062000EB9FF5F0EA9E42F0E99D42F0E89C45F030
:0106300022A7
:10063100E8600FECC313FCED13FDEE13FEEF13FFA7
:03064100D8F122CB
:0C064400ECF0A3EDF0A3EEF0A3EFF02229
:10065000A8828583F0D083D08212066712066712C3
:100660000667120667E473E493A3C583C5F0C583E8
:10067000C8C582C8F0A3C583C5F0C583C8C582C8F4
:010680002257
:0C068100A42582F582E5F03583F5832284
:06068D008A838982E473F8
:10005E00E5702432F582E4346FF583E0057022906A
:10006E006F2F300903906F32E475F0011206B30260
:10007E0003BA2002E97F2ED2028018EF540F24908B
:10008E00D43440D4FF30060BEF24BFB41A00500313
:10009E002461FFE571600215710574E57470020547
:1000AE007330090E906F2FE475F0011206B3EF0254
:1000BE00069302303E7403D2098003E4C209F57040
:1000CE00906F2F1206CAE4F571F573F574E5716041
:1000DE00077F201200A180F5F572C203C202C2048E
:1000EE00C205C207C208C20A12006DFF700D3009A8
:1000FE00057F001200B2AF74AE7322B42561C2D573
:10010E00C20612006DFF24D0B40A00501C75F00A0E
:10011E0020D50DC571A42571F5717002D20580E050
:10012E00C572A42572F57280D724CFB41A00EF5091
:10013E0004C2E5D2060202ACD20380C4D20280BE53
:10014E00D20480BAD2D580B8D20780B27F201200F6
:10015E00A12004077401B5710040F112005EFF1278
:10016E0000A10200DBD20AD208809312005EFB12BD
:10017E00005EFA12005EF94A4B700679787A037BBC
:10018E00FF200433E571602FAF72BF00011F7E00A8
:10019E008E827583001203D360050EEE6F70F1C26E
:1001AE00D5EBC0E0EAC0E0E9C0E0EE1202F0D0E02C
:1001BE00F9D0E0FAD0E0FB1203BAFF60A5EBC0E085
:1001CE00EAC0E0E9C0E01200A1D0E02401F9D0E0DD
:1001DE003400FAD0E0FBE57260DDD572DA80837B05
:1001EE00FF7A0279ECD2048098791080027908C2E5
:1001FE0008C20A8008D2D5790A8004790AC2D5E4E9
:10020E00FAFDFEFF12005EFC7B0820031312005E57
:10021E00FD7B1030020A12005EFE12005EFF7B2094
:10022E00EC3382D592D55013C3E43002069FFFE41F
:10023E009EFEE42003039DFDE49CFCE4CBF8C20388
:10024E00EC700CCFCECDCCE824F8F870F38017C349
:10025E00EF33FFEE33FEED33FDEC33FCEB33FB9966
:10026E004002FB0FD8E9EB300305F8D0E0C448B2EA
:10027E0003C0E00AEC4D4E4F78207B0070C2EAC0FE
:10028E00E01202F2D0F0D0E0200304C4C0E0C4B209
:10029E0003C0F012008AD0F0D5F0EB0200DB12069C
:1002AE00D301795301F758014A4C01464201FB4FE5
:1002BE00020344020349015F4302095501ED460161
:1002CE00ED4501ED47039B50014E2D01522E017558
:1002DE002B01562301732003862A0000016D3F3F38
:1002EE003F00790AA2D5200514300709B91002047F
:1002FE0004B9080104A2D5200802500104200466A6
:02030E00920457
:10031000B571005032C0E07F203005177F30A20455
:1003200072087207500D120347C204C208C2077F49
:1003300030800F300703E9C0E01200A1300703D07E
:10034000E0F9D0E0B571CE3007177F30B9100C124C
:1003500000A17F583006077F788003B90803120098
:10036000A13004057F2D0200A17F20200AF87F2BF9
:100370002008F322920480CF286E756C6C29002D22
:1003800050434958D20312005E3003F8C20378711B
:1003900030D504D2027872F602010C12005E2403FA
:1003A000B405004001E490037F93120092743A1266
:0A03B0000092D2057571040201F7F6
:102F2C00EFC394094006EFC3940E4004EFB42003A2
:052F3C00D38001C32257
:102C9300EFC394414006EFC394474018EFC39461D8
:102CA3004006EFC39467400CEFC394304009EFC371
:092CB300943A5003D38001C322BE
:10253400906F0EEBF0A3EAF0A3E9F0906F11E0FBCB
:10254400A3E0FAA3E0F91203BAFE906F0EE0FBA336
:10255400E0FAA3E0F91203BAFD6E702AED600E9062
:102564006F1474FFF5F01204C145F070037F00226C
:10257400906F0FE475F0011204C1906F12E475F0CE
:10258400011204C180B5D3EE6480F8ED64809840F4
:07259400037F01227FFF22FB
:102E0600E94A4B7001221203BAFF6D700122EF707E
:0C2E160004FBFAF92209E970ED0A80EAD9
:10161800906F28EBF0A3EAF0A3E9F0906F28E0FBC5
:10162800A3E0FAA3E0F91203BAFF122F2C500C9092
:101638006F29E475F0011204C180E0D201906F288F
:10164800E0FBA3E0FAA3E0F91203BAFF642B6004FD
:10165800EFB42D1D906F28E0FBA3E475F001120490
:10166800D7A9F0FA1203BA642D6003D38001C3929C
:1016780001906F2B12065000000000906F28E0FBCD
:10168800A3E0FAA3E0F91203BAFF122FA1506A7F70
:101698000A7E007D007C00906F2BE0F8A3E0F9A3A0
:1016A800E0FAA3E0FB1204EDC8ECC8EDC0E0EEC020
:1016B800E0EFC0E0906F28E0FBA3E0FAA3E0F912A6
:1016C80003BAFF3395E0FEEF24D0FFEE34FFFEE4CB
:1016D800FCFDD0E0FBD0E0FAD0E0F9EB2FFFEA3ECA
:1016E800FEED39FDEC38FC906F2B120644906F2903
:1016F800E475F0011204C18082300110906F2BE074
:10170800FCA3E0FDA3E0FEA3E0FF8011906F2BE0B7
:0E171800FCA3E0FDA3E0FEA3E0FF1206A52265
:10069300BB010689828A83F0225002F722BBFE0146
:0206A300F32240
:0E06A500C3E49FFFE49EFEE49DFDE49CFC2266
:1006B300F8E0FBA3A3E0F925F0F0E58215827002D0
:0706C3001583E0FA38F02274
:0906CA00EBF0A3EAF0A3E9F02231
:1006D300D083D082F8E4937012740193700DA3A3B6
:1006E30093F8740193F5828883E4737402936860CA
:0606F300EFA3A3A380DFCA
:102FA100EFC394304009EFC3943A5003D38001C377
:012FB10022FD
:00000001FF
